:10000000031E080085015F30A000213084008001BC
:10001000840AA00B07282F2824208400073984068F
:100020000310840C840C840C041A841704128419A1
:10003000841684118A01820701340234043408349E
:10004000103420344034803407398A018207283440
:1000500029342A342B342C342D342E342F340730C9
:10006000B6001930B9217830B600FF30B92101301F
:10007000A9210230A9210330A9210430A92105308A
:10008000B4210830B4210130AD210530AD21083054
:10009000AD21A10101305F22FF308D213608A30080
:1000A000392101305F22FF308D213608A2006430F3
:1000B000BD212208422223083222031D502801308C
:1000C0005F22FF308D213608A20022084222230839
:1000D0003222031D5028220842222308FE2136081E
:1000E000A500250842220330D4213608A5002508A2
:1000F00042220230EB213608A5000530B121013043
:100100005F22FF308D213608A100210842222208FB
:100110002322031D7D280530AD21C830BD21A60155
:1001200001305F22FF308D213608A3002A30532290
:10013000422200302822031D0D29210842220130CD
:1001400002223608A1003230BD212108422232307D
:100150002D22031DAD283021A1012A305322422235
:1001600000302822031D0D296430BD2101305F229B
:10017000FF308D213608A2002208422223081E22C9
:10018000031DC3288F28220842222308FE21360897
:10019000A4002408422225082322031DD1288F28E9
:1001A0008F282608422201302822031DE9281F211A
:1001B0000130B7002C30BE211F210130B7002C3098
:1001C000BE211F210130B7002C30BE210130A60016
:1001D000B4282621A501A4012A305322422200304E
:1001E0002822031D0D290130BD2124304522013074
:1001F000022224304C22243045222730B90010300E
:100200002922031D0A292C305322422201302822A0
:10021000031DEC282B218F288A212B212C305322DF
:10022000422201302822031D0E290530B121013060
:10023000B700F430BE210530AD218F28642A083084
:10024000B1211930BD210830AD21642A0530B1211A
:100250000830B121642A0530AD210830AD21642A6F
:100260000530B1216430BD210530AD216430BD21A0
:10027000642A0530B1213230BD210530AD21323044
:10028000BD210530B1213230BD210530AD213230E4
:10029000BD210530B1213230BD210530AD213230D4
:1002A000BD210530B1213230BD210530AD213230C4
:1002B000BD210530B1213230BD210530AD213230B4
:1002C000BD210530B1213230BD210530AD213230A4
:1002D000BD210530B1213230BD210530AD21323094
:1002E000BD210530B1213230BD210530AD21323084
:1002F000BD210530B1213230BD210530AD21323074
:10030000BD210530B1213230BD210530AD21323063
:10031000BD21642A0730CB218A29B8005B22B22193
:100320000A30BD213A088004841380068413000833
:100330003A050319A7293A088417800600008006A9
:100340003808B707031C9629B60F9629B603B701DC
:10035000642A0C2084178004642A0C20FF3A80054C
:10036000B6290C208004B5290C20FF3A841780059B
:10037000642A840036088000642AB701B60010227F
:1003800064003708360403190800F730FF3E031DE8
:10039000C6291222C0298316F83881050F39810435
:1003A00063000F308104642AB901B8001030BF0027
:1003B000BE01BD010314B60DB70DBD0DBE0D162255
:1003C0003D300522031C361016223D30361C052216
:1003D000BF0BDA29642AB901B8003D304C22B701BD
:1003E000B6013E083D040319642A0310BE0CBD0C7F
:1003F000031804220310B80DB90DF129B901B80092
:100400001622042AB901B800363084003808800763
:100410003908840F00000318013E031C8007642A7A
:10042000B709B609B60A0319B70A08001B22B80AA9
:100430000319B90A642AB909B809642AB901B800CC
:1004400037220139642AB901B80037220339642AF6
:10045000B901B80037220239642AB901B80037223D
:100460000539642AB901B80037220639642A3908E7
:100470003702031D3F2A3808360203190234031CD1
:1004800004340134B701B600642A84000008B600C1
:10049000840A0008B700642A840036088000840AB1
:1004A00037088000642A0D20BD000005841B3D062E
:1004B0000319003401343B0884003A080800242062
:0E04C0000D20BA000408BB008312640008007F
:02400E00DC3F95
:00000001FF
